:10000000830100308A003028A00003088301A30088
:100010000B1C0B280C281B28051815280F2810303E
:100020002202031815281428172816281B28A101B6
:10003000A10A1030A20083120C1C1F2820282A2895
:10004000A10B2328242826288312D723CF308312FC
:100050008F070C10831223088300A00E200E0900C6
:1000600021308400233039208301B52B0406800120
:0A007000840A0406031D362800343C
:10075A0085010B1383168C018B1163008312080029
:10076A00FF2383169000FD3085007F3081009501BC
:10077A00950A8312850183169601960A8B11073012
:10078A008312990083160C148C018C0A3030831260
:10079A00900410140B17A201A101A10A8B17D52BE3
:1007AA00D52B3028220883169B001C141A088312A2
:1007BA00A100A108031DE22BE32BF12B2208123A18
:1007CA00031DE82BE92BEA2BAD2383169B011C148E
:1007DA001A088312A100A2018312A11FF52BF62B7E
:1007EA00F82B8514FA2B831285108312A113A20AFF
:0407FA00831208005E
:02400E00843FED
:10420000320084000300830004008100010081006B
:10421000010081006E006E00000000000000000040
:10422000010081000000000000000000000000000C
:00000001FF
